:020000040800F2
:100000004008002045010008C31F0008511D0008DA
:10001000C11F0008890B00087123000800000000C0
:10002000000000000000000000000000B5200008F3
:100030008B0B000800000000C51F0008B720000857
:100040005F0100085F0100085F0100085F01000810
:100050005F0100085F0100085F0100085F01000800
:100060005F0100085F0100085F0100085F010008F0
:100070005F0100085F0100085F0100085F010008E0
:100080005F0100085F0100085F0100085F010008D0
:100090005F0100085F0100085F0100085F010008C0
:1000A0005F0100085F0100085F0100085F010008B0
:1000B0005F0100085F0100085F0100085F010008A0
:1000C0005F0100085F0100085F0100085F01000890
:1000D0005F010008652300085F0100085F01000858
:1000E0005F0100085F0100085F0100085F01000870
:1000F0005F0100085F0100085F0100085F01000860
:100100005F0100085F0100085F0100085F0100084F
:100110005F0100085F0100085F0100085F0100083F
:100120005F0100085F0100085F0100085F0100082F
:10013000DFF80CD000F0F8FC00480047E14100086F
:10014000400800200648804706480047FEE7FEE7D3
:10015000FEE7FEE7FEE7FEE7FEE7FEE7FEE7FEE777
:100160001721000831010008202A04DB203A21FA77
:1001700002F00021704721FA02F3D040C2F12002C0
:10018000914008431946704740EA01039B0703D09A
:1001900009E008C9121F08C0042AFAD203E011F8C6
:1001A000013B00F8013B521EF9D27047D2B201E088
:1001B00000F8012B491EFBD270470022F6E710B56C
:1001C00013460A4604461946FFF7F0FF204610BDC5
:1001D000F0B480EA0102D40F4200B2EB410F02D228
:1001E0000246084611464A0042D0C30DDDB2C1F3B3
:1001F000C752AD1A202D35DAC1F3160141F40002C1
:1002000004B15242C5F1200602FA06F12A41104417
:10021000B3EBD05F23D0C4B1012DA0EBC35009DCF8
:10022000F0BC4FF0004202EAC352DBB200F500001E
:1002300000F0F5BA400000F1807000EBC350A0F16F
:10024000807040EAD170490009E0490841EAC07174
:10025000A0EBC35000F50000400800EBC350F0BC19
:1002600000F0D4BA6142012202EB4101001BF6E723
:10027000F0BC704781F00041AAE780F00040A7E79A
:1002800080EA010210B502F00043400022D04A008B
:100290001FD0010E01EB1261C0F35600C2F35602EB
:1002A00040F4000042F40002A0FB022000047F3969
:1002B000140400D0401C50EA124001D44000491EF2
:1002C000C2B20C0604EBD010401C4008802A02D0B9
:1002D00003E0002010BD20F00100002900DA00201A
:1002E000184310BD30B480EA010202F0004530F03E
:1002F000004221F0004013D090B1C30DD40DC2F3E1
:100300001601C0F31600E41A41F4000140F40002A3
:100310007D34914201D3641C00E04900002C02DAD4
:1003200030BC002070474FF400000023914201D3FD
:10033000891A034340084FEA4101F7D151B1914274
:1003400002D14FF0004105E002D24FF0010101E07F
:100350006FF0010103EBC450284430BC00F056BAE2
:10036000420005D0C0F3C7525242914201DC002046
:10037000704700EBC15070472DE9FE4F804681EA7F
:100380000300C00F0C46009021F0004123F000450F
:10039000B8EB0200A94105D24046214690461C46D2
:1003A0000B46024623F00040104347D0270DC7F309
:1003B0000A00C3F30A510290401A019040286BDAF8
:1003C000C3F3130040F4801B0098924620B1002331
:1003D000D2EB030A63EB0B0B01985946C0F14002C4
:1003E000504600F0F2F906460D4650465946019A2D
:1003F00000F0FAF910EB08006141002487EA11527D
:1004000084EAE7731A4340D0009A62B3019A012A42
:100410004FEA075215DC001B61EB02014FF000426E
:1004200002EA0752CDE90042001C41F58011324634
:100430002B4600F060FA03B0BDE8F08F404621463D
:10044000F9E7001B61EB0201001C41F58013001865
:100450005B412018A2F5001747EB030140EAD57075
:10046000B6196D4111E06D084FEA360645EAC075D0
:100470004FEA0752001B61EB0201001C41F580119D
:1004800049084FEA30000019514132462B4603B06B
:10049000BDE8F04F00F020BA009801224000002390
:1004A000D0EB020263EBE073009821464FEAE07460
:1004B000B8EB000061EB0401E9E783F000435BE780
:1004C00081F0004158E72DE9FE4F81EA030404F072
:1004D000004421F0004100944FF0000B23F0004352
:1004E00050EA01045ED052EA03045BD0C3F30A541D
:1004F000C1F30A552C44A4F2F3340194A0FB025436
:10050000C1F3130141F48011C3F3130343F48013C7
:1005100001FB024400FB034E840A970A44EA81541B
:1005200047EA8357A4FB076802958D0A05FB0785F8
:100530004FEA932C04FB0C542705029D4FEA065802
:1005400047EA1637B5EB08056EEB070C870E920EDF
:1005500047EA811742EA8312A7FB0201B6EB0B01BF
:1005600064EB00042B0D43EA0C335E1844EB1C5083
:10057000DA465146E7FB0201C5F313044FEA0B3399
:1005800043EA14534FEA0432019C43EA0603A4F100
:100590000C040294009CCDE900B400F0ACF903B067
:1005A000BDE8F08F00200146F9E770B521F0004367
:1005B00003430CD0C1F30A550024D5EB040564EBCA
:1005C0000403D617AD1AB34102DB0020014670BD0B
:1005D000201841EB025170BDC10F80EAE070084461
:1005E000CA079623002100F01AB99623002211466B
:1005F00000F015B900F0004220F00040C10DC0F33A
:10060000160040F400007F2901DA00207047962987
:1006100003DCC1F19601C84001E096398840002A08
:10062000F4D04042704720F00040C10DC0F31600E6
:1006300040F400007F2901DA00207047962903DC8E
:10064000C1F19601C840704796398840704770B52F
:10065000C1F30A5201F000450024C1F3130140F236
:10066000FF3341F480119A4201DA002070BD40F25C
:1006700033439A42A2F2334203DC5242FFF774FD45
:1006800000E090402C43F1D0404270BD00F00042A9
:1006900030F000400AD0C10D01F56071C0F31600C2
:1006A00042EA0151C2084007114370470020014649
:1006B0007047000030B5041E71F1000404DB4FF0F8
:1006C0000044404264EB0101141E73F1000405DB99
:1006D0001C464FF00043524263EB04038B4208BFB9
:1006E000824230BD30B5041E71F1000404DB4FF0CE
:1006F0000044404264EB0101141E73F1000405DB69
:100700001C464FF00043524263EB0403994208BF7A
:10071000904230BD002801DBC0F10040002901DB20
:10072000C1F1004181427047002801DBC0F1004067
:10073000002901DBC1F100418842704730B50B460A
:10074000014600202022012409E021FA02F59D4201
:1007500005D303FA02F5491B04FA02F52844151ED5
:10076000A2F10102F1DC30BD2DE9F05F0546002069
:1007700092469B4688460646814640241BE0284612
:10078000414647462246FFF7EFFC53465A46C01AF9
:10079000914110D311461846224600F016F82D1A42
:1007A00067EB01084F4622460120002100F00DF8BA
:1007B00017EB00094E41201EA4F10104DFDC48467E
:1007C00031462A464346BDE8F09F202A04DB203A02
:1007D00000FA02F1002070479140C2F1200320FA94
:1007E00003F3194390407047202A06DBCB17203AC9
:1007F00041FA02F043EAE07306E041FA02F3D04026
:10080000C2F1200291400843194670470029A8BF51
:100810007047401C490008BF20F00100704710B429
:10082000B0FA80FC00FA0CF050EA010404BF10BCDE
:10083000704749B1CCF1200421FA04F411FA0CF10B
:1008400018BF012121430843A3EB0C01CB1D4FEA44
:1008500000614FEA102042BF002010BC704700EB3F
:10086000C35010440029A4BF10BC7047401C49006D
:1008700008BF20F0010010BC7047F0B4002802DC73
:10088000F0BC00207047C0F3C751C0F3160040F41D
:100890000000CA0701D14000491E3F2202EB61055A
:1008A000002211464FF4000626FA01F31344D4182F
:1008B000844201D8001B1A464000491C1729F3DD69
:1008C0005100814202D24FF0FF3100E0002102EBE3
:1008D000C550F0BCFFF79ABF10B5141E73F10004A9
:1008E00008DA401C41F1000192185B411A4301D122
:1008F00020F0010010BD2DE9F04D92469B4611B14C
:10090000B1FA81F202E0B0FA80F220329046FFF7AD
:100910005CFF04460F4640EA0A0041EA0B015346D9
:100920005A46084313D0114653EA010019D0C8F1C2
:1009300040025046FFF718FC05460E465046594601
:100940004246FFF742FF084305D0012004E020465D
:100950003946BDE8F08D0020054346EAE0762C4399
:1009600037430A986305E40AA0EB08000022FD0A59
:1009700044EA47540A3002D500200146E9E7010560
:1009800010196941DDE9084500196941BDE8F04DDC
:10099000A2E72DE9F04D81EA030404F0004B21F0B9
:1009A000004514464FF0000A23F0004150EA0502CA
:1009B00020D054EA01021DD0C5F30A570246C5F300
:1009C0001303C1F31300C1F30A5640F4801543F436
:1009D0008013A7EB0608101BD64608F2FD3873EB10
:1009E000050002D308F1010801E092185B41B8F15B
:1009F000000F03DA00200146BDE8F08D00204FF41F
:100A00008011064684460EE0171B73EB050705D3DD
:100A1000121B63EB050306434CEA010C49084FEA3D
:100A2000300092185B4150EA0107EDD152EA030011
:100A300012D082EA040083EA0501084305D0101BA6
:100A4000AB4106D20122002306E000224FF0004312
:100A500002E06FF0010253101AEB06004CEB085154
:100A600010EB0A0041EB0B01BDE8F04DFFF734BF7E
:100A70002DE9F041054621F000400C46284309D0FD
:100A8000C4F30A5040F23341884205DD284621462E
:100A9000BDE8F0812846FBE740F2FE31884210DCD9
:100AA0000CDB4FEA043040EA155050EA053105D01E
:100AB000104804F0004101430020E9E7002001460E
:100AC000E6E7A0F233404642C6F1400228462146FE
:100AD000FFF77BFE07468846284621463246FFF749
:100AE00043FB43463A46FFF7F7FE3246BDE8F04186
:100AF000FFF76BBE0000F03FC1F30A52C1F31301D0
:100B000040F2FF3341F480119A4202DA002001469C
:100B1000704740F233439A42A2F2334202DC52421F
:100B2000FFF722BBFFF751BE064C074D06E0E06819
:100B300040F0010394E8070098471034AC42F6D324
:100B4000FFF7FAFAA0500008C05000080EB5C10F18
:100B500080EAE0700844CA07002140F233438DE880
:100B60000E000A460B46FFF7C6FE03B000BD0EB5E9
:100B700040F2334102910021CDE900110A460B46B3
:100B8000FFF7B9FE03B000BDFEE7704772B6FEE79F
:100B900030B585B000241848009401940294039461
:100BA000816941F004018161816901F004010491CE
:100BB000816941F008018161816901F008010491B6
:100BC000816941F01001816180690C4D00F01000D5
:100BD000049000221021284600F0DCF9102000903B
:100BE0000120CDE90104022003906946284600F067
:100BF000D5F805B030BD00000010024000080140EB
:100C000010B590F821100022022905D0042181633B
:100C100080F82020012010BD01680B6823F00E032E
:100C20000B6001680B6823F001030B6090F8403003
:100C3000C46B012101FA03F3636080F8211080F88E
:100C40002020104610BD00002DE9F05F90F8211023
:100C50000024022903D004218163012485E0016876
:100C60000A6822F00E020A6001680A6822F0010296
:100C70000A603F4E3E4FB215DFF8F4C0DFF8F09047
:100C8000DFF8ECA0DFF8E8B0DFF8E4E00168783FD7
:100C900013011502ACF1640CA9F15009AAF13C0A48
:100CA000ABF1280BAEF1140E4FF48018B14227D9E6
:100CB000B9420ED0614512D049451DD0514518D0DA
:100CC000594518D0714501D1424615E0294EB1422F
:100CD00001D1012210E0274E1436B14201D1102279
:100CE0000AE0244E2836B14206D0224A3C329142D4
:100CF00001D11A4600E02A461E49091F0A602BE06E
:100D0000B94213D0614517D0494522D051451DD075
:100D100059451DD0714501D142461AE0B14202D178
:100D20004FF0807215E0134EB14201D1012210E064
:100D3000104E1436B14201D110220AE00D4E283671
:100D4000B14206D00B4A3C32914201D11A4600E032
:100D50002A46074980394A60012180F82110002184
:100D600080F82010416B01B188472046BDE8F09F14
:100D7000800002400804024070B5044600F010F9FB
:100D80000546601C02D004480078044400F008F9CD
:100D9000401BA042FAD370BD040100202DE9F84F9A
:100DA000DFF8C8910024A9F1040B23460F2709F1AD
:100DB000040AABF1040ED1E00125A54006EA0502C4
:100DC000AA4276D1DFF8A8C14E68A6EB0C086645AA
:100DD0002BD00DDC032E34D005DC36B3012E19D018
:100DE000022E2FD11BE0112E16D0122E2AD119E07F
:100DF000B8F5881F19D006DCB8F5803F15D0B8F5D6
:100E0000801F1FD111E0B8F5001F0ED0B8F5041FE8
:100E100018D10AE0CB6815E0CB681B1D12E0CB6847
:100E200008330FE0CB680C330CE08B682BB1012B3F
:100E30004FF0080303D0456104E0042302E005619C
:100E400000E00023FF2A01D8064601E000F1040675
:100E50004FEA840501D9A5F12005D6F8008007FAEC
:100E600005FC28EA0C0803FA05F548EA0508C6F867
:100E700000804D68ED0070D53E4DAE6946F001062C
:100E8000AE61AD6924F0030605F0010500953A4D09
:100E900006EB050CDCF80850A607360F07FA06F833
:100EA00025EA0805DFF8D480404503D14FF000085B
:100EB00025E052E0DFF8C880404502D14FF001083C
:100EC0001DE0DFF8C080404502D14FF0020816E077
:100ED000DFF8B480404502D14FF003080FE0DFF89F
:100EE000AC80404502D14FF0040808E0DFF8A08054
:100EF000404502D14FF0050801E04FF0060808FA1E
:100F000006F848EA0508CCF808804D68D9F8006072
:100F1000ED024D4601D5164300E096432E604D6824
:100F2000DAF80060AD02554601D5164300E096435D
:100F30002E604D68DBF80060AD035D4601D51643B9
:100F400000E096432E604D68DEF80060ED037546C4
:100F500001D5164300E096432E60641C0A681646CD
:100F6000E2407FF429AFBDE8F88F0000080401409B
:100F70000000111000100240000001400008014074
:100F8000000C014000100140001401400018014015
:100F9000001C01400AB1016170470904FBE7000031
:100FA0000148806870470000040100200248816801
:100FB000027811448160704704010020074810B591
:100FC000016841F010010160032000F06DF80F206E
:100FD00000F006F800F024F8002010BD00200240C8
:100FE00070B50D4D04464FF47A712878B1FBF0F0DE
:100FF0000A490968B1FBF0F000F060FC48B9102C18
:1010000007D200222146501E00F02EF800206C600E
:1010100070BD012070BD00000401002010010020FF
:10102000094808B5816941F001018161816901F0D8
:1010300001010091C16941F08051C161C06900F0B6
:101040008050009008BD000000100240002809DB1D
:1010500000F01F02012191404009800000F1E020D2
:10106000C0F8001170470000F0B40E4B1B680C462E
:10107000C3F30223C3F10705042D00D90425191D6C
:10108000072901D2002300E0DB1E012606FA05F144
:10109000491E214099409E40761E16403143F0BCC7
:1010A00001F08CB90CED00E0064900F00702086879
:1010B0004FF6FF03184040EA0220034A104308603D
:1010C000704700000CED00E00000FA052DE9F04744
:1010D0000F46050061D0434E306800F00700B8426B
:1010E00009D2306820F0070038433060306800F0E3
:1010F0000700B84251D128683B4C810712D5400700
:1011000003D5606840F4E06060602878000703D58C
:10111000606840F4605060606068A96820F0F0008A
:10112000084360602878C00728D06868012810D07C
:101130002168022810D0890700292EDA616821F081
:10114000030101436160FFF72BFF804641F28839BC
:101150000DE021688903EFE78901EDE7FFF720FF44
:10116000A0EB0801494502D90320BDE8F08760687B
:10117000696800F00C00B0EB810FEFD1306800F02F
:101180000700B8420BD9306820F0070038433060C0
:10119000306800F00700B84201D00120E5E7287868
:1011A000400705D56068E96820F4E06008436060A6
:1011B0002878000706D56068296920F4605040EA65
:1011C000C100606000F038F86168084AC1F303119B
:1011D000515CC8400649086006480068FFF700FFF8
:1011E0000020C2E70020024000100240664F0008C5
:1011F00010010020080100200448054900684968E2
:10120000044AC1F30221515CC8407047100100201C
:1012100000100240764F00080448054900684968FC
:10122000044AC1F3C221515CC8407047100100203C
:1012300000100240764F00080E4A51680E4801F037
:101240000C03042B11D0082B0FD10C48C1F383439E
:10125000C903C05C0AD55168084AC1F34041921ED7
:10126000515C054A5043B0FBF1F0704704494843D4
:10127000704700000010024000127A00564F00082C
:1012800000093D002DE9F84F040070D02078C04DD2
:10129000C00749D06868C0F38100012807D068689A
:1012A000C0F38100022809D16868C00306D5286808
:1012B000800339D560680028E7D035E06068B0F574
:1012C000803F0BD010B1B0F5A02F11D0286820F4CA
:1012D00080302860286820F4802002E0286840F4EC
:1012E00080302860606890B1FFF75AFE06460AE039
:1012F000286840F480202860F0E700BFFFF750FE28
:10130000801B642873D828688003F7D50CE0FFF7AA
:1013100047FE064605E000BFFFF742FE801B64283B
:10132000F0D828688003F7D420789A4E80074FF0D1
:1013300001094FF0000839D5686810F00C0F07D08C
:101340006868C0F38100022809D16868C00306D428
:101350002868800714D52069012808D110E0206989
:10136000B0B1C6F80090FFF71BFE074605E00AE1A2
:10137000FFF716FEC01B0228C4D828688007F7D5DF
:101380002868616920F0F80040EAC10028600DE09B
:10139000C6F80080FFF704FE074604E0FFF700FEF2
:1013A000C01B022823D828688007F7D420780007BC
:1013B0002CD57948A169D9B1C0F80090FFF7F0FDAC
:1013C000074604E0FFF7ECFDC01B02280FD8686A4F
:1013D0008007F7D571484FF4FA510068B0FBF1F07F
:1013E000009000BF0098411E0091FAD20EE080E00C
:1013F000C0F80080FFF7D4FD074604E0FFF7D0FDFA
:10140000C01B022875D8686A8007F7D42078400787
:1014100060D5E8690027C00008D4E86940F0805032
:10142000E861E869012700F0805000905C4801689D
:10143000C90513D40168834641F480710160FFF748
:10144000AFFD824606E000BFFFF7AAFDA0EB0A0051
:1014500064284ED8DBF80000C005F5D5E068012807
:101460000AD008B1052813D0286A20F001002862AC
:10147000286A20F0040002E0286A40F00100286297
:10148000E06841F2883B98B1FFF78AFD82460BE0A5
:10149000286A40F004002862EEE700BFFFF780FDF5
:1014A000A0EB0A0159455AD8286A8007F6D50CE006
:1014B000FFF776FD824605E0FFF772FDA0EB0A011B
:1014C00059454CD8286A8007F6D41FB1E86920F046
:1014D0008050E861E06988B36968C1F3810102293D
:1014E00044D00228C6F8608004D0FFF759FD0446B6
:1014F00038E034E0FFF754FD074604E0FFF750FD05
:10150000C01B02282BD828688001F7D4206AB0F5C8
:10151000803F05D16868A16820F400300843686006
:10152000D4E908010843696821F47411084368602C
:10153000C6F86090FFF734FD044606E025E000BFE2
:10154000FFF72EFD001B022809D828688001F7D577
:101550001BE000BFFFF724FD001B022802D9032077
:10156000BDE8F88F28688001F4D40EE00128F7D098
:101570006868226A00F48031914204D1616A00F403
:101580007010884201D00120EAE70020E8E700005F
:10159000001002400000424280044242100100203C
:1015A0000070004070B5040009D0606A002540B1A9
:1015B00025616561A56294F8510040B10CE00120FD
:1015C00070BD6068B0F5827FF4D0E561F2E784F821
:1015D0005050204600F040F8022084F85100206866
:1015E000016821F040010160A088218900F4827027
:1015F00001F404410843A18901F400610843217CFE
:1016000001F002010843217D01F001010843218B13
:1016100001F400710843217F01F03801084394F878
:10162000201001F080010843218D01F4005108438E
:1016300021680860A069042101EA1040216848601F
:101640002068C16921F40061C1616565012084F8E9
:101650005100002070BD000030B585B0002400941A
:1016600001940294039400681549884225D11548D5
:10167000C16941F48041C161C16901F480410491B3
:10168000816941F00801816180690F4D00F0080017
:1016900004904FF42040009002200190032003901A
:1016A00069462846FFF77AFB4FF48040CDE90004F5
:1016B000694628460294FFF771FB05B030BD000073
:1016C0000038004000100240000C01402DE9FF4F9F
:1016D00081B01D46934604464FF001090E9EFFF768
:1016E0005FFC074694F851006168012806D0B1F507
:1016F000827F3CD1A168C9BB042838D10298002858
:1017000071D0BBF1000FFBD0002DF9D094F8500040
:1017100001282CD04FF0010A84F850A094F8510011
:10172000042802D0052084F851004FF00008C4F8C6
:101730005480C4F838B0E587A58702992163E5860F
:10174000A586C4F84080C4F8448020680168490632
:1017500003D4016841F040010160E068B0F5006F1A
:10176000606808D0F0B3012D49D081E0FFE7022086
:1017700005B0BDE8F08F08B1012D39D1206B21688B
:101780000088C860206B801C2063E08E401EE086CD
:101790002EE02068816889070FD5E18E69B1B9F123
:1017A000010F0AD1216B0988C160206B801C206366
:1017B000E08E401EE0864FF0000920688168C9076E
:1017C0000CD0E18F51B1C068A16B0880A06B801C68
:1017D000A063E08F401EE0874FF00109FFF7E0FBB8
:1017E000C01B01E00BE067E0B04201D3701C50D198
:1017F000E08E0028CDD1E08F0028CAD13EE0206BDA
:10180000216800780873206B401C2063E08E401E26
:10181000E0862DE02068816889070FD5E18E69B1E7
:10182000B9F1010F0AD1216B09780173206B401CBB
:101830002063E08E401EE0864FF00009206881683A
:10184000C9070CD0E18F51B1C068A16B0870A06BC3
:10185000401CA063E08F401EE0874FF00109FFF7B6
:101860009FFBC01BB04202D3701C01D011E086B1B7
:10187000E08E0028CED1E08F0028CBD13A46314609
:10188000204600F0A0FB50B12020606584F8508015
:1018900012E084F851A084F85080032068E7A06823
:1018A00018B92068C1688068009084F851A084F855
:1018B0005080606D0028F1D0012059E710B5401E1E
:1018C000B0F1807F01D3012010BD4FF0E0246061B2
:1018D0000F21601700F072FD0020A0610720206139
:1018E000002010BD70477047F8B5016804460868CD
:1018F000CA684B6910F00F0F4FF000055AD003F083
:10190000010602F49077374365D0C10705D0D105B1
:1019100003D5616C41F001016164410705D5D90728
:1019200003D0616C41F002016164810705D5D907DC
:1019300003D0616C41F004016164010707D502F036
:101940002001314303D0616C41F008016164616C96
:1019500000293BD0800604D5900602D5204600F031
:101960000AFC20684069616CC0F3801001F0080136
:10197000014320462BD000F0D7FB20684069400689
:1019800021D52068143050E8001F21F0400140E8C4
:101990000012002AF5D1E06BA8B16D494163E06BFC
:1019A000FFF752F9002811D0E06B416B01B0BDE8A0
:1019B000F040084783060ED593060CD52046BDE8B7
:1019C000F84000F0D8BB2046FFF78DFFF8BDFFF7C9
:1019D0008AFF6564F8BD266B2023012E7CD1C606E4
:1019E0007AD5D60678D508684868009048694FF0DF
:1019F0000206400640D5E16B086840680004000C10
:101A0000E8D0A28D8242E5D9E085886920282DD0D2
:101A100020680C3050E8001F21F4807140E800126B
:101A2000002AF5D12168143151E8000F20F001009F
:101A300041E80002002AF5D12068143050E8001F68
:101A400021F0400140E80012002AF5D184F842302C
:101A5000256320680C3050E8001F21F0100140E899
:101A60000012002AF5D1E06BFFF7CAF86663A08D7B
:101A7000E18D401A81B22AE0A08DE18D401A81B239
:101A8000E08D0028A6D00029A4D022680C3252E8AC
:101A9000000F20F4907042E80007002FF5D1206875
:101AA000143050E8002F22F0010240E80027002FF8
:101AB000F5D184F84230256320680C3050E8002FBF
:101AC00022F0100240E80023002BF5D16663204687
:101AD000FFF708FFF8BDFFE705062BD5150629D54A
:101AE00094F841002128F5D1A068B0F5805F01D1BC
:101AF0002069B0B1206A411C2162216800784860E9
:101B0000E08C401E0004000CE084E3D12068C16832
:101B100021F08001C1602068C16841F04001C160CE
:101B2000D8E7206A0088C0F308004860206A801C5B
:101B30002062E5E74006CDD55006CBD5CA682046E1
:101B400022F04002CA6084F8413000F000F9C1E799
:101B50001921000870B5040004D094F84100002554
:101B600010B106E0012070BD84F84050204600F01E
:101B700023F8242084F841002068C16821F4005132
:101B8000C160204600F058FB2068016921F49041B3
:101B900001612068416921F02A0141612068C16822
:101BA00041F40051C1606564202084F8410084F84C
:101BB00042006563002070BD2DE9F04786B0002526
:101BC0000646009501950295039532490068324C0E
:101BD0000F154FF002084FF00309884231D1E06938
:101BE00040F48020E061E06900F480200490A06966
:101BF00040F01000A061A069DFF8A0A000F0100084
:101C0000CDE90390CDE9007869465046FFF7C6F864
:101C1000E014CDE90005694650460295FFF7BEF88D
:101C20001F48416821F0300141F0E06141F01001AE
:101C30004160002211462720FFF716FA2720FFF700
:101C400005FA18493068884220D1A06940F48040E4
:101C5000A061A06900F480400490A06940F00400F5
:101C6000A061A069104C00F0040004904815CDE973
:101C700000086946CDF80C902046FFF78FF8CDE9B3
:101C80000075694620460295FFF788F806B0BDE862
:101C9000F0870000004800400010024000100140A2
:101CA00000000140003801400008014070472DE964
:101CB000F843044690F84100984616460D46202801
:101CC00002D00220BDE8F88385B17EB100206064B7
:101CD000212084F84100FFF763F9A6848146E68459
:101CE000A0682027B0F5805F02D003E00120E9E77B
:101CF000206910B12E4600250EE000260CE0802160
:101D0000204600F0F5FAA8B9C6B116F8010B216813
:101D10004860E08C401EE084E08C4B464FF00002AF
:101D2000CDF800800028EAD14FF04001204600F0B5
:101D3000DFFA40B184F841700320C3E735F8020BA5
:101D4000C0F30800E3E784F841700020BAE7704769
:101D5000FEE7000010B500F02FF8002002F06CFE46
:101D600001221149752000F0B3F80F480178472986
:101D700005D00EA000F0FEFA6FF0020010BD0F219A
:101D80004E2003F0B3F8002802DA6FF0030010BD14
:101D9000002002F021FE0028F9DB002002F05AFEAC
:101DA0000028F4DB012010BD440200204944203DFE
:101DB000202578200A0D000010B5002002F03CFE1E
:101DC0000121112003F092F8BDE810400120FEF738
:101DD000D3BF000010B5FFF7BDFF04000FD522A050
:101DE00000F0C8FA26A000F0C5FA21462CA000F0A9
:101DF000C1FA21A000F0BEFAFFF7ACFFFCE72CA06F
:101E000000F0B8FA05220020304902F089FE0120D6
:101E100002F054FE012002F065FE0621002002F0CF
:101E200073FC0121002002F025FC01220221002088
:101E300002F092FF01220F21002002F02FFF062165
:101E4000012002F061FC0121084602F013FC072288
:101E50000221012002F080FF0122BDE810400F2185
:101E6000104602F01BBF0000494D55B3F5CABCBB7C
:101E7000AFB2BBB3C9B9A620200D0A2000000000F4
:101E8000BCECB2E9494D55BDD3CFDFBBF2B3A2CA1A
:101E9000D4D1ADBBB7B9A9B5E720200D0A20000009
:101EA000B4EDCEF3D7B4CCAC3A256420202020008A
:101EB0000D0A202049434D34323638385F496E6967
:101EC0007420CDEAB3C9200D0A0000000000F03FE5
:101ED000F8B514460F4605460F2A02D94FF0FF30D9
:101EE000F8BD144E002210213046FFF753F8124877
:101EF00045F0800100F8011B2146FEF75EF9FF2046
:101F00000D4A0090631C10320B490C48FFF7DEFBB2
:101F100010B16FF00100F8BD012210213046FFF72B
:101F200039F80549224611313846FEF72DF90020CF
:101F3000F8BD0000000801404000002028030020F8
:101F4000104810B50E4901604FF4827141600021C4
:101F500002228160C0E90312012242615202C0E9FB
:101F600006210162416281620A21C162FFF71AFB08
:101F7000002803D0BDE81040FEF708BE10BD0000E9
:101F800000380040280300200C4810B50A490160C1
:101F90004FF4E1314160002181600C22C160C0E951
:101FA00004128161C161FFF7D5FD002803D0BDE8AF
:101FB0001040FEF7EBBD10BD00380140800300204B
:101FC000FEE7FEE77047F8B515460E460B46009251
:101FD00004460122022100F011F840B933460022E4
:101FE00080212046009500F009F8002804D0606D9B
:101FF00040F0200060650320F8BD00002DE9F843A3
:102000001E46914688460446089DFEF7C9FF401BC0
:10201000351AFEF7C5FF074625480068C0F3CB30E8
:10202000684338E0701C37D0FEF7BAFFC01BA842E7
:1020300003D215B1009860B32CE02068416821F00C
:10204000E00141606068B0F5827F0BD1A068B0F517
:10205000004F02D0B0F5806F04D12068016821F0F4
:1020600040010160A06AB0F5005F09D120680168F5
:1020700021F4005101602068016841F400510160C1
:10208000012084F85100002084F850000320BDE8AE
:10209000F8830025401E00902068816838EA01001E
:1020A00004D000214945BDD10020F0E70121F9E726
:1020B000100100207047FEF779BF30B58FB028219E
:1020C0006846FEF77AF814210AA8FEF776F802258A
:1020D0000120049000951020059000244FF460101A
:1020E000CDE9084007956846FFF7CCF808B172B60D
:1020F000FEE70F20CDE90A054FF48060CDE90C40E2
:1021000002210AA80E94FEF7E1FF002801D072B662
:10211000FEE70FB030BD704710B5406A0021C185A1
:10212000C184FFF7E0FB10BD01680C3151E8002FBE
:1021300022F4907241E80023002BF5D1016814319C
:1021400051E8002F22F0010241E80023002BF5D1D5
:10215000016B012909D101680C3151E8002F22F0EF
:10216000100241E80023002BF5D1202180F8421015
:1021700000210163704708B590F84210222901D070
:10218000022008BD82684FF480539A4201D1016950
:1021900021B1816A9A421BD04AB10AE00268816A81
:1021A0005268C2F308020A80816A891C08E0026949
:1021B00072B10268526802F07F020A70816A491C9B
:1021C0008162C18D491E0904090CC18503D01BE041
:1021D00002685268F1E70168CA6822F02002CA600A
:1021E0000168CA6822F48072CA6001684A6922F0F4
:1021F00001024A61202180F8421000214163026BF4
:10220000012A03D0FFF752FD002008BD01630168D9
:102210000C3151E8002F22F0100241E80023002B7E
:10222000F5D101680A68D20602D50A6849680091AA
:10223000818DFFF757FBE7E770B504460068016939
:10224000E26821F44051114301612169A06808430B
:10225000616908432168CA6841F20C639A430243EA
:10226000CA6020684169A26921F44071114341614B
:102270001E492068884202D1FEF7CEFF01E0FEF73A
:10228000BBFF00EBC00101EB00126068642180001D
:10229000B2FBF0F3B3FBF1F36FF018067343B2FB3C
:1022A000F0F5B2FBF0F605EB8305322303EB0515E1
:1022B000B5FBF1F5B6FBF1F605F0F00505EB0615FB
:1022C000B2FBF0F6B2FBF0F0B0FBF1F06FF01802E9
:1022D000504306EB800003EB0010B0FBF1F02168E7
:1022E00000F00F002844886070BD000000380140F5
:1022F0002DE9F843984617460D460446089E24E00B
:10230000701C22D0FEF74CFEA0EB0800B0421AD899
:10231000CEB12068C168490717D5802D15D0402D52
:1023200013D00168C94309070FD40168002540682C
:1023300000902046FFF7F8FE0820606484F84050C3
:102340000120BDE8F8830320FBE72068006835EA38
:10235000000004D00020B842D2D00020F1E70120D4
:10236000F9E700000148FFF7BFBA00008003002032
:10237000FEE700000FB4054B10B503A9044A02980C
:1023800000F024FC10BC5DF814FB0000613800086C
:1023900014010020490050EAC12018BF04204A0D52
:1023A00018BF40F0010040F2FF72B2EB515F08BF6E
:1023B00040F00200012808BF052070470907090EF8
:1023C000002804DB00F1E02080F80014704700F0E2
:1023D0000F0000F1E02080F8141D70472DE9F74F41
:1023E000144694B00021C4E902111599079121F017
:1023F0000045C9498D4206DC1599C4E9000117B0B2
:102400000020BDE8F08FC549DFF814A3A9423CDDE8
:102410000799C44E0029C44FC44A1599534619DD83
:10242000FEF74BF8554506D0C14AC24BFEF745F8BA
:10243000C4E900010AE04FF0D352BE4BFEF73DF86D
:1024400032463B46FEF739F8C4E9000117B00120D7
:10245000BDE8F08FFDF790FF554506D0B44AB54B67
:10246000FDF78AFFC4E900010AE04FF0D352B14BF7
:10247000FDF782FF32463B46FDF77EFFC4E90001CF
:1024800017B04FF0FF30BDE8F08FAB49A942159966
:1024900078DB21F0004183468846A84AA84BFEF726
:1024A00012F80022A74BFDF767FFFEF7D0F809905E
:1024B000FEF74CFB06460F469C4A5346FEF703F8D0
:1024C00043465A46FDF7FCFF80468A46984A994B98
:1024D00030463946FDF7F7FF2A0D01250B9242469B
:1024E0005346FDF7EDFF032DC4E9000139D00B98E9
:1024F000C1F30A51401A05EB45111139814230DA16
:102500009148C346784400EB0510CDF80CA00C9020
:10251000D0E9002330463946FDF7D5FF02460B4689
:102520000491069058460399FDF7C7FF80468A46F6
:1025300002460B4658460399FDF7BFFF049B069AD7
:10254000FDF7BBFF83460C9803913946D0E902237F
:102550003046FDF7B8FF5A46039BFDF7AEFF6D1CF2
:10256000BDE707980028A2BF099817B0BDE8F08F13
:10257000616881F000416160099817B04042BDE890
:10258000F08FFFE784461598C1F31301C0F30A509A
:10259000A0F2F5304FEA601800F01F06C6F12000E7
:1025A000139000200690079041F4801E05206D4690
:1025B00076B1664A08EB00017A4452F8213002EB0A
:1025C0008101B3404A68139922FA01F1194305E0E9
:1025D0005F4908EB0002794451F82210A1FB0E2755
:1025E000A1FB0C131A449A4234BF0123002303EBCE
:1025F000070A05EB8003D3E901B70F448F4234BFCC
:102600000121002193448B4411B1934502D903E089
:10261000934501D2012100E00021C3E901B75144F3
:1026200045F82010011EA0F10100C1DC0298059FB1
:1026300000F10050800F12900298DDE903568000EF
:10264000FEF784FA834628460D91FEF790FA6FF064
:102650001D02FDF7AAFFCDE90E013046FEF787FA0D
:102660006FF03D02FDF7A1FF80468A463846FEF72F
:102670007EFA6FF05D02FDF798FF0746424653462B
:102680001191FDF779FEDDE90E23FDF775FE5A463F
:102690000D9BFDF771FE00250E465A4628460D9B00
:1026A000FDF70BFFDDE90E23FDF707FF424653461A
:1026B000FDF703FF3A46119BFDF702FFDFF898A0F4
:1026C000244A5346FDF7FFFE07468846234A244B1B
:1026D00031462846FDF7F7FE3A464346FDF74CFEE5
:1026E000074688464FF0A842534631462846FDF734
:1026F000EAFE3A464346FDF73FFE159A12F0004FB8
:1027000004D0129A81F0004152421292C4E90001B1
:10271000129817B0BDE8F08FFB21E93F7CD9024049
:10272000FB21F93F7370032E8A19A33B000040542C
:102730003163621A61B4D03DFB21394183C8C96D50
:10274000305FE43F0000E03FA82A0000242A000098
:10275000062A0000182D4454FB21F93D3326A6110A
:10276000460B113C2DE9FF4D21F0004807460C4671
:10277000B8F1795F08DAFDF76AFF002801BF002091
:10278000324904B0BDE8F08D3A462346104619465A
:10279000FDF799FE054602462D480E460B460621DA
:1027A000784400F05DF82A463346FDF78CFEDDE9FB
:1027B000022382468B4638462146FDF784FE0446B6
:1027C0000F4652465B4628463146FDF77CFE2246C0
:1027D0003B46FDF772FE07468A464FF0FF32284619
:1027E0003146FDF7E2FE1B4A90450ADA3A46534667
:1027F000FDF763FE04B00022BDE8F04D134BFDF77A
:102800005FBE154A4245A8BFA8F500154FF0000469
:10281000B8BF124D22462B46FDF74FFE06468846AE
:1028200022462B4600200949FDF747FE04460D4687
:102830003A46534630464146FDF73FFE04B0224635
:102840002B46BDE8F04DFDF73BBE00000000F03F19
:10285000DC2700003333D33F0000E93F0000D23FC4
:102860002DE9F0414F1E00EBC7010446D1E90001FC
:1028700015461E4637F006020DD02A463346FDF7B0
:1028800022FE7F1E04EBC703D3E90023FDF774FD8E
:1028900037F00602F1D1022F25D0042F13D0062FD6
:1028A00018BFBDE8F0812A463346FDF70CFED4E997
:1028B0000A23FDF761FD2A463346FDF704FED4E9FD
:1028C0000823FDF759FD2A463346FDF7FCFDD4E900
:1028D0000623FDF751FD2A463346FDF7F4FDD4E902
:1028E0000423FDF749FD2A463346FDF7ECFDD4E904
:1028F0000223FDF741FD2A463346FDF7E4FDD4E906
:102900000023BDE8F041FDF737BD00002DE9FF4D84
:10291000054621F0004084B00C46B0F1795F0BDA37
:102920002846FFF737FD042808BF00F06FF8284657
:1029300008B02146BDE8F08D2A460B461046FDF74B
:10294000C2FD06460F462A462346FDF7BCFD8046DB
:1029500026488A4632463B4605217844FFF780FFE9
:1029600083461098029160B3214A224B404651465B
:10297000FDF7A9FDCDE900015A4640465146029BAC
:10298000FDF7A1FD82468846DDE906014FF0FF32E2
:10299000FDF70BFE52464346FDF78FFD32463B46A0
:1029A000FDF791FDDDE90623FDF787FDDDE9002355
:1029B000FDF783FD08B02A462346BDE8F04DFDF73C
:1029C0007FBD0B465A4630463946FDF77CFD084A26
:1029D000084BFDF7D1FC42465346FDF774FD08B0A5
:1029E0002A462346BDE8F04DFDF7C6BC1A27000075
:1029F000495555555555C5BF0122FDF7D6BD002295
:102A0000134610461146FDF7C4BF0000024A0020DD
:102A10001107FDF7CABD000001FDFFFF02E008C875
:102A2000121F08C1002AFAD170477047002001E048
:102A300001C1121F002AFBD1704700000149086044
:102A400070470000180100202DE9FF5F82B00021CF
:102A5000DDE90430020DDDF840B0034318D044F640
:102A60001050A2F2FF3242431514119801281FD0D2
:102A7000A5EB0B00401C5FEA000A4FF000064E4F2A
:102A8000DFF83891B046504615D5CAF1000413E07E
:102A9000119801244AA3012801D16FEA0B01029881
:102AA000119AC0E90031C0E9024206B0BDE8F09FCA
:102AB000CBF10000DFE704460021404A491842EB11
:102AC0000450CDE9001012E0E00707D032463B4643
:102AD00040464946FDF7F7FC8046894632463B466C
:102AE00010461946FDF7EFFC06460F466410002C11
:102AF000EAD1DDE90401DDE90023BAF1000F06DACD
:102B0000FDF7E1FC42464B46FDF7DDFC05E0FDF735
:102B100040FF42464B46FDF73CFF04460E4600226E
:102B2000284BFDF7DFFD03D84FF0FF30014607E0EB
:102B30000022254B20463146FDF71EFCFDF7DCFF49
:102B4000102409E0002C0ADB0A220023FDF70CFE0A
:102B5000039B30321A55641E50EA0102F2D1641C04
:102B6000039AC4F111031444119A012A03D00122DB
:102B700008430DD10AE0084304D000204FF0110BA8
:102B8000119072E7A3EB0B056D1E0DE05B4504DDB4
:102B90004FF0000205F1010504E003DA4FF00002F6
:102BA000A5F10105002AECD002981199C0E9023183
:102BB000C0E9004579E70000000014400000F03F44
:102BC000300000000000F0430000E03F2DE9FF4F1F
:102BD00095B09B468946064600250FE2252877D109
:102BE00000242746F84A0121059400E0044316F822
:102BF000013F203B01FA03F01042F7D130782A2838
:102C000011D06FF02F033078A0F13002092A16D8C6
:102C1000059A44F0020402EB820203EB42021044E4
:102C2000761C0590EFE759F8042B0592002A03DA89
:102C3000504244F40054059044F00204761C30786D
:102C40002E2816D116F8010F44F004042A280DD0BE
:102C50006FF02F023078A0F13003092B09D807EB71
:102C6000870302EB4303C718761CF3E759F8047B8C
:102C7000761C30786C280FD006DC4C2817D06828DA
:102C80000DD06A2814D104E0742810D07A280FD10E
:102C90000DE044F400140AE044F4801401E044F42C
:102CA00040147278824202D104F58014761C761C9E
:102CB000307866280BD013DC582877D009DC002840
:102CC00075D04528F6D04628F4D047281AD19DE182
:102CD00018E0632835D0642879D0652812D195E1B1
:102CE000702873D008DC6728F1D069286FD06E286F
:102CF0000DD06F2806D1B5E073282CD0752875D07B
:102D0000782874D05A46179990476D1C75E1C4F322
:102D10000250022809D003280DD0D9F80010042849
:102D20000DD00D6009F1040967E1D9F80010EA1728
:102D3000C1E90052F6E7D9F800100D80F2E70D70F6
:102D4000F0E719F8041B8DF8001000208DF8010041
:102D5000EA46012003E059F804AB4FF0FF30610769
:102D60004FF0000102D40DE008F101018846B9429C
:102D70000FDA8045F8DB1AF808100029F4D108E0D2
:102D800008F1010188468142FADB1AF8081000298F
:102D9000F6D105985B46A0EB080721463846179AFE
:102DA00000F094FA284400EB080507E04DE029E123
:102DB0000DE01AF8010B5A4617999047B8F101082F
:102DC000F7D25B4621463846179A13E142E00A22C1
:102DD0000092C4F302524FF0000A022A08D059F8B8
:102DE00004CB032A4FEAEC710AD00DE029E02AE077
:102DF00009F1070121F00702F2E802C1914609E05A
:102E00000FFA8CFC4FEAEC71042A03D14FFA8CFCC8
:102E10004FEAEC71002907DA0A460021DCF1000CC8
:102E200061EB02012D2202E0220504D52B228DF850
:102E30000420012203E0E20701D02022F7E79046B8
:102E400059E00A2102E010220DE010214FF0000AA3
:102E500000910BE010224FF0000A44F00404082710
:102E6000009203E008224FF0000A0092C4F30252DD
:102E7000022A05D059F804CB0021032A08D009E022
:102E800009F1070121F00702F2E802C1914605E0CD
:102E90001FFA8CFC042A01D10CF0FF0C4FF0000843
:102EA000220728D5702806D0009B83F0100353EA30
:102EB0000A0305D00EE040228DF80420012208E02C
:102EC0005CEA010206D030228DF804208DF805005E
:102ED00002229046009B83F0080353EA0A030AD1BA
:102EE0005CEA010201D1620705D530228DF8042089
:102EF0004FF001087F1E582804D034A003900EA87C
:102F000002900DE036A0F9E753466046009AFDF7BF
:102F10002BFC84460398825C0298401E029002704B
:102F20005CEA0100F0D1029806A9081A00F1200A13
:102F3000600702D524F4803400E00127574502DD04
:102F4000A7EB0A0000E0002000EB0A0100900598C2
:102F50004144401A0590E00306D45B462146179A87
:102F6000059800F0B3F90544002706E001A85A4689
:102F7000C05D179990476D1C7F1C4745F6DBE00349
:102F80000CD55B462146179A059800F09FF9054439
:102F900004E030205A46179990476D1C0099481E4E
:102FA00000900029F5DC08E0029802995A46007862
:102FB000491C0291179990476D1CBAF10001AAF1C2
:102FC000010AF1DC65E100000928010030313233EB
:102FD0003435363738396162636465660000000055
:102FE000303132333435363738394142434445463F
:102FF0000000000000F058F90544761C30780028E5
:103000007FF4ECAD19B02846BDE8F08F620700D41C
:10301000062709F1070222F0070CFCE80223E1462B
:1030200003F000485FEA080C02D00FF2702C0DE0AC
:103030005FEA045C02D50FF2682C07E05FEAC47C0B
:1030400002D00FF2602C01E0AFF2700C4FF0FF38AD
:1030500023F00043CDF850C065280CD006DC45288D
:1030600009D046281DD047283DD13DE0662818D01C
:1030700067287ED138E00021112F01DB112000E00C
:10308000781CCDE9000106A90EA8FFF7DDFCDDE9FB
:103090000F010E9A03910021009207F1010A049199
:1030A0004DE04FF000400097CDE9011006A90EA8B1
:1030B000FFF7CAFCDDE90F0203920E9B1199002273
:1030C000DDF80CA00093049211B9791C00EB010A01
:1030D000B7EB0A0004D4C0F1FF3007F1010A0490F5
:1030E000AAEB0700019044E0012F00DA012700213C
:1030F000112F01DD112000E03846CDE9000106A9BD
:103100000EA8FFF7A1FCDDE90F010E9A0391002143
:1031100004910092BA4621070CD40399514500DA74
:103120008A46BAF1010F05DD009AAAF10101515C4E
:10313000302908D0B84202DA10F1040F06DA012172
:10314000CDE9011015E0AAF10101E9E7002805DC4D
:10315000049901440491AAEB000102E0411C51458D
:1031600000DD8A460499401A401C01904FF000404F
:103170000290200704D40198504501DBCDF804806B
:1031800000208DF84F0002980DF14F07B0F1004F6D
:1031900025D02B200E9002984FF0020800280CDA60
:1031A000404202902D200E9007E00A210298FDF780
:1031B000C5FA3031029007F8011DB8F10001A8F1FD
:1031C0000108F2DC02980028EFD1791E0E980870F1
:1031D000307800F0200040F0450007F8020D12A8FA
:1031E000C01B00F107081498007800B1012000EB23
:1031F0000A01019801EBE07105984144401A401E14
:103200000590E00306D45B462146179A059800F026
:103210005DF805441498007818B15A4617999047FC
:103220006D1CE00324D55B462146179A059800F0F3
:103230004DF805441CE00498002807DBDDE9030194
:10324000884203DD0098405C179901E0179930200F
:103250005A469047049805F10105401C04900198D6
:10326000401E019004D12E205A46179990476D1C9C
:10327000BAF10001AAF1010ADDDC05E017F8010B43
:103280005A46179990476D1CB8F10001A8F1010842
:10329000F4DC5B462146179A0598ABE62D0000004A
:1032A0002B000000200000002DE9F041044600251D
:1032B0001E461746880404D405E039462020B0474E
:1032C0006D1C641EF9D52846BDE8F0812DE9F0415A
:1032D000044600251E469046C80301D5302700E06D
:1032E0002027880404D505E041463846B0476D1CC8
:1032F000641EF9D52846BDE8F081000070B50024B1
:10330000FDF791F90B4E054604EBC400AAB206EB9B
:103310008000C82100F05FF9641C032CF4DB054831
:103320004FF4C8715C38A0F85010002141650120AD
:1033300070BD0000840100202DE9FC47284D814626
:103340002868FDF757F9274C20806868FDF752F987
:103350006080A868FDF74EF9A08021460222084649
:1033600000F07AF82049486D012830D020888A89F9
:10337000A31D801A02B21A806088CD89401B05B255
:103380005D80A088098A401A04B29C801046FDF72F
:1033900023F96FF00B084146FCF7E2FF124E074697
:1033A0000C3E30602846FDF717F94146FCF7D8FF80
:1033B000054670602046FDF70FF94146FCF7D0FF47
:1033C000B060C9E90075C9F80800BDE8FC8720684D
:1033D000A188ADF804100199BDE8FC4700F014BFC6
:1033E00014020020000000202801002070B50546CE
:1033F00020F0004613493046FCF742FF1249FCF723
:10340000E7FE3146FCF73CFF1049FCF7E1FE314690
:10341000FCF736FF0E49FCF7DBFE044631464FF061
:103420007E50FCF727FF01F04BFD2146FCF728FFFB
:1034300015F1FF4F05D3BDE8704001460548FCF784
:1034400019BF70BD306E99BC2716983D843459BEA3
:10345000A40DC93FDB0F494030B5B1F90040B1F9C7
:103460000230B1F90410921E072A05D2DFE802F0FB
:10347000070A0F13171A1D00048043801AE0038007
:10348000624202E0624202805A42428012E05A42A4
:10349000028044800EE062420280438009E00380A3
:1034A000448006E004805A4202E05A4202806242AE
:1034B00042804942818030BD2DE9F04721F000462D
:1034C00020F000450F46804629463046FDF72CF98E
:1034D00001D2344600E02C4614F0FF4F0CD02946B0
:1034E0003046FDF717F901D2304600E02846214664
:1034F000FCF7F8FE044600E0002422492046FCF7D1
:10350000BFFE2149FCF764FE2146FCF7B9FE4FF0EF
:103510007E51FCF75DFE81461C492046FCF7B0FE5B
:103520001B49FCF7A7FE2146FCF7AAFE1949FCF748
:10353000A1FE2146FCF7A4FE1749FCF79BFE21469D
:10354000FCF79EFE1549FCF798FE4946FCF7CAFEBB
:10355000044631462846FDF7E7F804D221461048D4
:10356000FCF788FE04460F4DAF4204D321460E48B7
:10357000FCF780FE0446A84501D384F000442046B1
:10358000BDE8F08799FB243F69A2163E39094E3DFC
:10359000E3B59E3E88FA163E45FE7F3FA7DFA8347E
:1035A000DB0FC93F00008080DB0F4940F8B50446BF
:1035B0001F4615460846069EFDF735F881B2AAB2A9
:1035C0003B462046009600F021F80020A061606193
:1035D0002062E061F8BDF8B5064615460F464FF08B
:1035E000804001F06DFC01464FF07E50FCF77AFE02
:1035F00004463846FCF7F9FF0146002000902346B8
:103600002A463046FFF7D2FFF8BD00002DE9F0470B
:1036100004461F460E461046DDF82080FCF7E5FF05
:1036200005463046FCF7E1FF3549FCF729FE2946FF
:10363000FCF726FE3349FCF723FE064601F0DCFBCF
:103640000546304600F0AEF8814601213846FCF7C9
:1036500087FE01462846FCF745FE06464FF04047E8
:103660004FF07E55B8F1000F06D0B8F1010F0ED023
:10367000B8F1020F18D137E049462846FCF7FAFDA9
:103680004FF0FF316060FCF76BFE206031E039469F
:1036900048462560FCF7F4FDC4E90105E0603146C9
:1036A0002846FCF7E7FD206129463046FCF790FDEF
:1036B000054629462068FCF715FE2060294660680B
:1036C000FCF710FE60602946A068FCF70BFEA060C6
:1036D0002946E068FCF706FEE06029462069FCF711
:1036E00001FE2061BDE8F0870020C4E9006086F09B
:1036F0000040A06039464846FCF7C2FDCEE7000016
:10370000DB0FC940BD37863500B5244B21F00042A0
:1037100087B09A42DCBF0022134629DD204B9A4233
:1037200008D140B94FF00100FFF788F9FFF767F9BA
:1037300007B000BD03DBFFF75FF907B000BD02AAC9
:10374000FEF74CFE10F0030104BF0DF1080C9CE8DD
:103750000F000DD0012001290ED0022914D00DF147
:10376000080C00909CE80F00FFF7D0F807B000BDF0
:10377000FEF7F8FF07B000BD0DF1080C00909CE8C3
:103780000F00FFF7C3F805E00DF1080C9CE80F00EF
:10379000FEF7E8FF07B081F0004100BDFB21E93FE3
:1037A0000000F07F10B50349FCF712FDBDE81040A2
:1037B00001F022BBDB0FC93F10B5FCF70DFFBDE8E0
:1037C00010400149FCF75CBD35FA8E3C00210161D7
:1037D00070472DE9F041044600690E46401C206107
:1037E000012820D0FCF7F8FE25688046294630469F
:1037F000FCF740FD07464146FCF774FD2946FCF7FF
:10380000E7FC0546606029463046FCF733FD01467B
:103810003846FCF735FDA168FCF7DAFCE06025606E
:10382000A060BDE8F081666000202660A060F8E737
:1038300010B500F004F8BDE8104001F041BB10B530
:1038400004460069012808DD401EFCF7C5FE01465C
:10385000E068BDE81040FCF745BD002010BD000049
:1038600038B504468DF8000002230122694602485B
:10387000FEF71DFA204638BD800300202DE9F04FE9
:1038800089B00E225B491D20FEF722FB002804DAD6
:103890004FF0FF3009B0BDE8F08F5649002001AA73
:1038A00031F810305BBA22F81030401C0728F7D3EB
:1038B000BDF90400FCF790FE4F4C2169FCF712FDA6
:1038C0006169FCF785FCA061BDF90600FCF784FE88
:1038D0000690216A0091FCF7D3FC464D543DD5F883
:1038E00000904946FCF7C6FC04F12806D6F8008093
:1038F0004146FCF7C5FC05F10C073860BDF908002E
:10390000FCF76AFE05900099FCF7BAFCD5F804B004
:103910005946FCF7AFFCD6F804A05146FCF7B0FCC2
:103920007860BDF90A00FCF757FE07900099FCF794
:10393000A7FCAD682946FCF79DFCB6683146FCF74C
:103940009FFCB86049460698FCF794FC4146FCF79A
:1039500097FC1837594638600598FCF78BFC5146A0
:10396000FCF78EFC786029460798FCF783FC31460B
:10397000FCF786FCB860BDF90C00FCF72DFE616A0F
:1039800082468B46FCF77CFC07F124042768394605
:10399000FCF770FCA4F130052860BDF90E00FCF7BF
:1039A0001BFE81465946FCF76BFC66683146FCF706
:1039B00061FC6860BDF91000FCF70EFE80465946B8
:1039C000FCF75EFCA4682146FCF754FCA860504656
:1039D0003946FCF74FFC1835314628604846FCF75D
:1039E00049FC686040462146FCF744FCA860012081
:1039F00050E70000440200200C00002070B50C4984
:103A00004FF4FA72A1F85020002214464A65FCF7E0
:103A10000AFE084E054604EBC400AAB206EB80007D
:103A2000C821FFF7D8FD641C032CF4DB012070BD16
:103A3000A4000020D40300202DE9FC478046FFF7B6
:103A40001DFF2E4D00280CDB2D4C2068FCF7D2FD0D
:103A500028806068FCF7CEFD6880A068FCF7CAFD8E
:103A6000A880264902220846FFF7F6FC2349254C88
:103A70000C31486D01282ED028888A898B1F801A26
:103A800002B21A806888CE89801B06B25E80A88840
:103A9000098A401A05B29D801046FCF79DFDDFF8AB
:103AA00068904946FCF71EFC074620603046FCF74C
:103AB00093FD4946FCF716FC064660602846FCF775
:103AC0008BFD4946FCF70EFCA060C8E90076C8F8FB
:103AD0000800BDE8FC87A9882868ADF804100199A2
:103AE00000F0D0FB002020606060A060C8F80000FB
:103AF000C8F80400C8F80800EBE7000098000020B0
:103B000020020020C80300206F1283412DE9FF5FCF
:103B1000444C61680F463846FCF7B2FB0390A1683D
:103B200000910846FCF7ACFBE16805468B46584619
:103B3000FCF7A6FB0646206839460446FCF7A0FBC6
:103B4000029020460099FCF79BFB8146594620468F
:103B5000FCF796FB804638460099FCF791FB8246BD
:103B600059463846FCF78CFB019059460098FCF703
:103B700087FB834601213046FCF7F2FB07463C46B3
:103B800001212846FCF7ECFB4FF07E5605463146F6
:103B9000FCF773FB2146FCF76DFB234C414620608C
:103BA0005046FCF767FB0121FCF7DAFB60604946F1
:103BB0000198FCF70DFB0121FCF7D2FBA060414608
:103BC0005046FCF705FB0121FCF7CAFBE060012130
:103BD0000398FCF7C5FB3146FCF74FFB0646394618
:103BE000FCF748FB206158460299FCF743FB012192
:103BF000FCF7B6FB606149460198FCF73BFB0121ED
:103C0000FCF7AEFBA06158460299FCF7E1FA0121EE
:103C1000FCF7A6FBE06129463046FCF72BFB20624F
:103C2000BDE8FF9F600000205402002010B50F2067
:103C3000FFF7C2FDFFF7B6FD02490863BDE810407B
:103C4000FFF764BF600000202DE9FF4F83B0884676
:103C50008146114616460846159FFCF711FB05469E
:103C600041460846FCF70CFB044649460846FCF76B
:103C700007FB2146FCF7ACFA2946FCF7A9FAFE4DF2
:103C8000FE4C8246002F7CD014990846FCF7F8FAC7
:103C9000139983460846FCF7F3FA1299074608463B
:103CA000FCF7EEFA3946FCF793FA5946FCF790FA1E
:103CB000A169002903DD491EA161F14901E04FF02E
:103CC0007E510091EF49884260DD00F07FFA07469F
:103CD00001461298FCF7D4FA129039461398FCF773
:103CE000CFFA834639461498FCF7CAFA1490A868AC
:103CF0001499FCF7C5FA019059466868FCF7C0FAB8
:103D0000074628681299FCF7BBFA3946FCF760FAB7
:103D10000199FCF75DFA074668691499FCF7B0FA57
:103D2000019059462869FCF7ABFA8346E868129976
:103D3000FCF7A6FA5946FCF74BFA0199FCF748FA4A
:103D400083460146FCF79CFA394601900846FCF789
:103D500097FA0199FCF73CFA01F0B2F8014658468F
:103D6000FCF78EFA80F000473946A869FCF788FA1C
:103D700001903946E869FCF783FA83463946286A98
:103D800000E01FE0FCF77CFA074603E000208346D2
:103D900007460190DDE90001FCF772FA4946FCF79D
:103DA00017FA814659460098FCF76AFA4146FCF733
:103DB0000FFA804639460098FCF762FA3146FCF764
:103DC00007FA0646069810F0FF4F07D1109810F03A
:103DD000FF4F03D1119810F0FF4F7DD01199084685
:103DE000FCF74EFA109983460846FCF749FA069903
:103DF00007460846FCF744FA3946FCF7E9F9594604
:103E0000FCF7E6F900F0E2F9074601460698FCF7F0
:103E100037FA069039461098FCF732FA1090394676
:103E20001198FCF72DFA1190D5F81CB05946FCF703
:103E300027FA00902F6A10983946FCF721FA00996A
:103E4000FCF718FA009039460698FCF719FAAD69A4
:103E5000074629461198FCF713FA3946FCF70AFA87
:103E6000019029461098FCF70BFA0546594606982A
:103E7000FCF706FA2946FCF7FDF9834983468A4593
:103E800035DA824F00983946FCF7FAF91699FCF7B3
:103E9000F7F9216AFCF79CF98246206239460198BD
:103EA000FCF7EEF91699FCF7EBF9616AFCF790F96B
:103EB0000546606239465846FCF7E2F91699FCF768
:103EC000DFF9A16AFCF784F90746A062514648462B
:103ED000FCF77EF9814600E034E029464046FCF7D5
:103EE00077F9804639463046FCF772F90646E069B4
:103EF000002803DD401E664DE06101E04FF07E5575
:103F0000644F00983946FCF7BBF92946FCF7B8F92D
:103F10004946FCF75DF9814639460198FCF7B0F94E
:103F20002946FCF7ADF94146FCF752F9804639467F
:103F30005846FCF7A5F92946FCF7A2F93146FCF7EB
:103F400047F906464FF0FF311698FCF709FA054687
:103F50004946FCF795F9039028464146FCF790F94D
:103F6000049028463146FCF78BF98346D4E901508A
:103F700026688146E068B24659460090FCF780F911
:103F8000804648460499FCF77BF9074685F00040D7
:103F90000399FCF775F93946FCF76CF94146FCF7D3
:103FA00069F93146FCF714F92060804604990098BD
:103FB000FCF766F9074659464846FCF761F906469C
:103FC00051460398FCF75CF93146FCF701F9394694
:103FD000FCF750F92946FCF7FBF8606007460099AA
:103FE0000398FCF74DF9019059462846FCF748F92B
:103FF000064650460499FCF743F93146FCF73AF976
:104000000199FCF7E5F84946FCF7E2F80646A0609E
:1040100049460398FCF734F9814628460499FCF791
:104020002FF9054659465046FCF72AF92946FCF770
:10403000CFF84946FCF71EF90099FCF7C9F801468C
:10404000E060FCF71DF9814631460846FCF718F997
:10405000054639460846FCF713F906464146084628
:10406000FCF70EF93146FCF7B3F82946FCF7B0F837
:104070004946FCF7ADF80FE0540200206000002034
:10408000000020410AD7233CE68AF93D6F12833AAB
:104090000000C842CDCCCC3E00F098F80546014661
:1040A0002068FCF7EDF8206029466068FCF7E8F826
:1040B00060602946A068FCF7E3F8A0602946E06844
:1040C000FCF7DEF8E06007B0BDE8F04FFFF71EBD7B
:1040D0002DE9F74F88B000210091D0E90321D0F8F5
:1040E00014B050F804AB8946F0E80571884690E8B2
:1040F000700012491046FCF7C3F807900F49484674
:10410000FCF7BEF881460D495846FCF7B9F80A9A03
:104110000099CDE9051202AB024683E87000CDE9B3
:104120000078494653460798FFF78EFD09980BB073
:104130000C30BDE8F04F00F003B8000035FA8E3CBB
:104140002DE9F0411B4C0646D4E90701FFF7B4F90D
:10415000194D2946FCF7C6F83060A06980F0004090
:10416000FFF744F91549FCF788F82946FCF7BAF837
:1041700070602168E068FFF79FF92946FCF7B2F804
:104180000F4FB0600F4DF86210F1FF4F03D30E498F
:10419000FCF71EF8B060206A396BFCF7C5FA286896
:1041A00002D240F0100001E020F010002860BDE8CD
:1041B000F08100005402002035FA8E3CDB0FC93F2D
:1041C00060000020000100200000B44310B500F0A2
:1041D00077FE0146BDE810404FF07E50FCF782B8F4
:1041E000FCF7ECFEFDF769FFFCF7D2FCFDF7A8FE3B
:1041F000FDF7CAFE00F06AF9024C204600F082F991
:10420000FBE700000AD7A33B2DE9F34100241C4D36
:10421000E8464FF4C8772646B5F85000B84208D1B2
:1042200004EB840005EB800045F824601430FFF7B0
:10423000CDFA55F8241038F91400084445F8240044
:1042400005EB44008681B5F8501001290ED155F8D0
:104250002410C83191FBF7F18181022C05D1084966
:10426000081D098AA1F5805181816E65641C032CAB
:10427000D2DB35F8500F401E2880BDE8FC810000DD
:10428000280100202DE9F34700243F4DEA46274648
:104290004FF4FA78B5F85000404508D104EB84009B
:1042A00005EB800045F824701430FFF78FFA55F8BD
:1042B00024103AF91400014445F82410FCF78CF955
:1042C000014604EB840005EB800014300646FFF73E
:1042D00080FA05EB44092DA0A9F80C70B5F8501030
:1042E000FEF748F8B5F85000012839D13046FFF7FD
:1042F0009FFA064621462CA0FEF73CF83046FCF714
:10430000C5F902460B462CA0FEF734F824A0FEF7B0
:1043100031F8B6F1814F32DC16F0FF4F2FD055F84F
:10432000241091FBF8F0A9F80C006F206F6585F858
:10433000580055F8241025A0FEF71CF8B5F90C100C
:104340002EA0FEF717F8B5F90E1031A0FEF712F8FF
:10435000B5F9101033A0FEF70DF811A0FEF70AF81A
:10436000641C032C96DBB5F85000401E0004000CC2
:10437000A5F8500001D1A5F85080BDE8FC87A5F84C
:10438000508001206865F8E7A40000202020206309
:1043900079636C65436F756E743A25642020202024
:1043A000200D0A2000000000202020617869733A67
:1043B0002564202020200000202020737464646580
:1043C000763A25662020202000000000202020676B
:1043D00079726F43616C6962726174696F6E2E6786
:1043E00079726F53756D2E617869735B617869734B
:1043F0005D3A256420202020000000002020206756
:1044000079726F5A65726F783A25642020202000F7
:104410002020206779726F5A65726F793A2564207F
:10442000202020002020206779726F5A65726F7AF1
:104430003A256420202020002DE9F04D07460E4645
:10444000FCF716FB04460D463A463346FCF738F8AF
:10445000DFF86CA0DFF86CB01B4B0746884616F0FF
:10446000004F4FF000020AD0FCF724F90AD90022CD
:104470005B4638464146FCF735F91BD212E0FCF7A3
:1044800019F908D20022534620462946FCF715F8B0
:1044900004460D460EE000225B4638464146FCF7D6
:1044A00021F907D80022534620462946FBF764FF2E
:1044B00004460D463146204665F31E01BDE8F08DE9
:1044C0000000F03F0000E03F0000E0BF70B5FDF7E6
:1044D00081FC094D2846FFF791FA084C20702846C8
:1044E000FEF70CFF217808402070FFF79FFBFCF7D8
:1044F00057FD0349886070BD0000FA439400002016
:104500001C03002070B505463D4CFCF749FD60607A
:10451000A168401AFCF769F83A49FBF7B1FE014679
:1045200020602846FCF7F6F869D86068A060A4F11E
:104530009800FFF781FAA4F1A400FEF7FDFEA4F1B4
:104540006C01A1F138002268FFF7C2FDA4F16C05EF
:10455000296B2869FBF78EFE2861E96AE868FBF79A
:1045600089FEE860FCF792F802460B4626A0FDF7AC
:1045700001FF2869FCF78AF802460B4625A0FDF7E3
:10458000F9FE6869FCF782F802460B4624A0FDF7A5
:10459000F1FE383D2868FCF779F802460B4622A068
:1045A000FDF7E8FE6868FCF771F802460B4621A0AB
:1045B000FDF7E0FEA868FCF769F802460B4620A06C
:1045C000FDF7D8FEE868FCF761F802460B461FA02D
:1045D000FDF7D0FE2869FCF759F802460B461EA0ED
:1045E000FDF7C8FE6869FCF751F802460B461DA0AE
:1045F000FDF7C0FE1EA0FDF7BDFE0020206070BDCF
:104600001C0300206F12833A726F6C6C3A2566208F
:104610000000000070697463683A2566200000009D
:104620007961773A25662000616363583A256620F0
:1046300000000000616363593A2566200000000015
:104640006163635A3A256620000000006779726F43
:10465000583A2566200000006779726F593A25663E
:10466000200000006779726F5A3A2566200000002A
:104670000D0A00002DE9F041224A137823F00206CA
:1046800043F0020550B1531C01281F7827F00104A4
:1046900047F001070FD0052822D019E0012908D0E2
:1046A00015700121762000F021FC164801780B20BE
:1046B0000CE01670F5E7012910D01F70022176205A
:1046C00000F014FC0F48401C0178032000F00EFCA1
:1046D000BDE8F0410021762000F008BC1C70EDE739
:1046E00001290BD015701F700121762000F0FEFB10
:1046F000044801780B2000F0F9FBDFE716701C700E
:10470000F2E700000F0000202DE9FC5F0C4601FBE2
:1047100004F96143090AE71F0191F91EA4F10E0B88
:10472000A4F11308A4F11B0AA4F12506A4F136058F
:10473000009140B3012873D0052872D10121762061
:1047400000F0D4FB21460C2000F0D0FB09F0FF0163
:104750000D2000F0CBFB9F48019A012C017862F3F9
:104760000301017075D0022C74D0032C73D0042C7B
:1047700072D0052C71D0062C6FD0032F6ED221F091
:10478000F0019031E7E00121762000F0AFFB2146F7
:104790000C2000F0ABFB09F0FF010D2000F0A6FBA0
:1047A0008C48019A012C017862F3030101700FD04B
:1047B000022C10D0032C12D0042C14D0052C16D0AF
:1047C000062C14D0032F16D221F0F00190313BE0DB
:1047D00041F0F00138E021F0F001D03134E021F077
:1047E000F001C03130E021F0F001B0312CE021F0D7
:1047F000F001A03128E0009A042A03D221F0F00150
:10480000803121E0BBF1050F03D221F0F0017031BE
:104810001AE0B8F1080F05D221F0F001603113E081
:104820001DE0D4E0BAF10A0F03D221F0F0015031BB
:104830000AE0102E03D221F0F001403104E0092DEE
:1048400003D821F0F00130310170624801780E2068
:10485000B5E046E048E04BE04EE051E054E0022194
:10486000762000F043FB5B48801C017864F346012E
:104870000170032000F03AFB09F0FF01042000F072
:1048800035FB5448019AC01C012C017862F30301E6
:10489000017067D0022C68D0032C6AD0042C6CD035
:1048A000052C70D0062C6ED0032F70D221F0F001B1
:1048B000903101707FE000BFBBF1050F6ED221F097
:1048C000F0017031F5E700BFBAF10A0F6DD221F0A7
:1048D000F0015031EDE7092D6DD821F0F0013031B4
:1048E000E7E741F0F00136E021F0F001D03132E0AD
:1048F00021F0F001C0312EE021F0F001B0312AE0CA
:1049000021F0F001A03126E0009A042A03D221F020
:10491000F00180311FE0BBF1050F03D221F0F0015F
:10492000703118E0B8F1080F03D221F0F0016031C6
:1049300011E0BAF10A0F03D221F0F00150310AE080
:10494000102E03D221F0F001403104E0092D03D8EC
:1049500021F0F001303101701E4801780E2000F086
:10496000C5FA7CE741F0F001A3E721F0F001D03176
:104970009FE721F0F001C0319BE721F0F001B03159
:1049800097E700E003E021F0F001A03191E7009A01
:10499000042A91D221F0F00180318AE7B8F1080FA2
:1049A00092D221F0F001603183E7102E93D221F0F2
:1049B000F00140317DE70748C01C0178052000F078
:1049C00095FABDE8FC5F0021762000F08FBABDE8C3
:1049D000FC9F00000E00002038B50446002000F0C7
:1049E0002BF8012269465020FDF772FA002802DAFE
:1049F0004FF0FF3038BD9DF8000064F35F10C1B286
:104A00008DF80010502000F071FA002802DA6FF0E3
:104A1000010038BDC4F1040101208840FBF7DCFD32
:104A20006FF00E01FBF79CFC014602480162C47264
:104A3000012038BD0C00002005490A78824201D1CE
:104A40000120704708700146762000F04FBA000040
:104A50000C00002038B504460020FFF7EDFF0122CE
:104A600069464F20FDF734FA002802DA4FF0FF3094
:104A700038BD9DF8000064F35F10C1B28DF80010DE
:104A80004F2000F033FA002802DA6FF0010038BD41
:104A90000120A040FBF7A0FD01460648FBF722FCE1
:104AA0006FF00E01FBF75CFC0146034841620473A2
:104AB000012038BD0000FA440C00002010B5044667
:104AC0000121762000F012FA012000EB0410C1B29F
:104AD000132000F00BFA0021BDE81040762000F012
:104AE00005BA00000D4910B50A78012812D042F02D
:104AF000010008700121762000F0F8F90748801EB7
:104B000001780B2000F0F2F90021BDE8104076207A
:104B100000F0ECB922F00100EBE700000F000020EC
:104B20002DE9F04704460E469046DFF850A1544D5B
:104B30000121762000F0DAF90022524B204631465E
:104B4000FBF7C1FC504A514BFBF7BDFC6FF0040270
:104B5000FBF72BFDFEF7D8FD0F46044621F0004180
:104B60000022A9462B46FBF7A5FD0BD808222046BC
:104B70003946FBF71AFDFFF75FFCFBF768FD05B24E
:104B800000262AE0012600224B4620463946FBF744
:104B9000A9FD09D222463B4600205146FBF78DFC79
:104BA0000322FBF702FD10E00022394B2046394674
:104BB000FBF780FD11D20022534620463946FBF711
:104BC000DBFB0022334BFBF77EFC0822FBF7EDFCFE
:104BD000FFF732FCFBF73BFD05B22F48B8F1000FA1
:104BE00009D0B8F1020F10D0B8F1040F17D0B8F106
:104BF000050F1CD03BE001782A0A66F3C30162F37B
:104C000000010170E9B20F202AE001782A0A66F358
:104C1000041162F341010170E9B2102020E0017833
:104C20002A0A66F3451162F38201017016E00178E9
:104C30002A0A66F3C30162F3000166F3041162F30A
:104C4000410166F3451162F382010170E9B20F2060
:104C500000F04CF9E9B2102000F048F9E9B2112057
:104C600000F044F90C480178122000F03FF9BDE84B
:104C7000F0470021762000F039B900000000F03F35
:104C80000000EC3F00408F401F85EB51B81E1940DB
:104C90000000ECBF000020C00D0000202DE9F04115
:104CA0000746002614460D463046FFF7C5FE17B1ED
:104CB000012F29D04BE00F2D01D8072C02D94FF03E
:104CC000FF3644E02348017865F3030164F347119C
:104CD00001704F2000F00AF9082C38D2DFE804F008
:104CE000370406080A0C0E1000200AE0012008E034
:104CF000022006E0032004E0042002E0052000E09A
:104D00000620FFF7A7FE22E00F2D01D8032C02D9C1
:104D10006FF001061BE00F48801C017865F303016A
:104D200064F347110170502000F0E0F834B1012C19
:104D300006D0022C06D0032C09D105E0002004E0A7
:104D4000012002E0022000E00320FFF745FE30468C
:104D5000BDE8F081140000202DE9F04707464FF030
:104D6000000815460E464046FFF766FE032E01D8A2
:104D70000F2D02D94FF0FF3838E01E48441C37B1E0
:104D800000F10309012F0DD0052F16D02EE0017878
:104D900066F383010170512000F0A8F8217865F3D3
:104DA00003011FE099F80010532066F3C40189F84D
:104DB000001000F09BF8217812E0017866F383017F
:104DC0000170512000F092F899F80010532066F31A
:104DD000C40189F8001000F089F8217865F3030117
:104DE00065F307112170522000F080F84046BDE8BD
:104DF000F08700001200002070B50446FBF7FAFBB4
:104E0000264D2030412807D3002070BD294620467A
:104E1000FBF730FA044600E0214EB442F6DC214EA6
:104E2000B44205D929462046FBF7D2F90446F7E7F4
:104E30001D498C4204DD0D462046FBF71BFA05E0B8
:104E40001A4DAC4206D92046FBF7C2F92946FBF7BA
:104E500014FA044621460846FBF712FA064614499E
:104E6000FBF70EFA1349FBF7B3F93146FBF708FAE3
:104E70001149FBF7ADF93146FBF702FA0F49FBF791
:104E8000A7F9054631462046FBF7FAF92946FBF714
:104E9000F7F92146BDE87040FBF79AB9DB0FC9402E
:104EA000DB0F4940DB0F49C0DB0FC93FDB0FC9BF38
:104EB0009A7C2E36FAAF4FB93587083CA4AA2ABE91
:104EC00070B50546FBF7D9FC044620F00040C0F160
:104ED000FF40C00F08D025F00040C0F1FF40C00FD8
:104EE00004BF0120FDF7AAFD204670BDF8B5154EA0
:104EF0000C460546002210213046FCF74BF81248BC
:104F000005F07F01104A017044704FF6FF70009069
:104F1000022310320C490D48FCF7D8FB0122102166
:104F20003046FCF737F8012209492846FCF7D0FF44
:104F300007480078A04201D10120F8BD4FF0FF30B2
:104F4000F8BD0000000801404000002028030020B8
:104F500044020020010202030405060708090A0BA7
:104F60000C0D0E0F101000000000000000000102E8
:104F70000304060708090000000001020304000002
:104F80004C5555555555A53F7751C1166CC156BF67
:104F90009015CB19A001FA3EAD529C804F7E92BE77
:104FA000C4B1B4BD9EEE213ED43888BEE9FAA8BD96
:104FB00000004054FB21F93F3163621A61B4D03DD7
:104FC0000000601A61B4D03D7370032E8A19A33BB0
:104FD0000000002E8A19A33BC14920259A837B3902
:104FE00000000000000000006E83F9A22915444E65
:104FF000D15727FCC0DD34F5999562DB4190433CE5
:10500000AB6351FE61C5BBDE3A6E24B7E0D24D42C0
:10501000EA2E49061C92D1091CEB1DFE3EA729B1C0
:10502000F53582E88444BB2E26709CE9417E5FB44E
:1050300039D69139F43953838B5F849C3B28F9BD71
:10504000FF97F81F0F9805DE8B112FEF1F6D0A5A7F
:10505000CF7E366DB709CB27663F464F2DEA5F9E60
:10506000C7BA27757BF1E5EBF739073DEA92528A1B
:10507000B15FFB6B085D8D1FA6F810111111813F08
:10508000D561C119A0012ABF7DFEB157E31DC73EFE
:10509000EB9C2B8AE6E55ABE7CD5CF5A3AD9E53D42
:1050A000C0500008000000201C0100001C2A00085D
:1050B000DC5100081C010020240700002C2A0008F5
:1050C00000000000000000000000000000000000E0
:1050D000000000000000000000000000E17A04432E
:1050E0000000C84100000000E803000000000000CC
:1050F000000000000000803F0000803F0000803F73
:10510000FF000000000000000000000000000000A0
:10511000FF00000000000000000000000000000090
:105120000000803F0000803F000000000000000001
:1051300000000000CDCC4C3E640000006400000084
:10514000000000000000000000000000000000005F
:10515000000000000000000000000000000000004F
:10516000000000000000000000000000000000003F
:10517000000000000000000000000000000000002F
:10518000000000000000000000000000000000001F
:10519000000000000000000000000000000000000F
:1051A00000000000000000000000000000000000FF
:1051B00000000000F40100000000000000000000FA
:1051C00000000000010000001000000000000000CE
:0C51D00000127A00000000000000000047
:0400000508000131BD
:00000001FF
